:0200000480007A
:100000006F00C00613000000130000001300000082
:100010001300000013000000130000001300000094
:10002000F32E003093FE0E08638A0E00B72E0000F8
:10003000938E0E8073900E3073002030F32E1034A8
:10004000938E4E0073901E3473002030B702002050
:10005000371300009303000203AE0200B382620074
:100060009383F3FFE39A03FE67800000130E1000F2
:1000700037050010930540061306500693066006E8
:100080002320D5002F26B518130710006318E61893
:10009000032705006394E618130E200037050010AF
:1000A0001305450093057006130680069306900617
:1000B0002320D5002F26B518130710006310E6166D
:1000C00003270500639CE614EFF05FF803270500A3
:1000D0006396E614130E3000370500101305450033
:1000E0009305700613068006930690062F26B51812
:1000F000130710006314E612032705006390E6124D
:10010000EFF0DFF403270500639AE610130E4000BA
:1001100037050010130585009305A0061306B006E9
:100120009306C0062320D500AF2705102F26B5184B
:100130006396D70E6314060E032705006390E50E41
:10014000EFF0DFF003270500639AE50C130E500073
:1001500037050010130585009305D0061306E00649
:100160009306F0062320D5002F26B5186308060A4B
:10017000032705006394E60AEFF05FED032705000F
:10018000639EE608130E7000370500101305450145
:1001900093058007130690079306A007930E0001AE
:1001A0002320D500AF2705102F26B5186398D70652
:1001B00063160606032705006392E506938EFEFF8D
:1001C00013054500938535001306360093863600E7
:1001D000E3980EFC130E9000370500101305051070
:1001E0009305B0071306C0079306D0072320D50058
:1001F000AF27051073000000AF27B51813070000E4
:10020000639EE70003270500639AE500EFF01FE413
:10021000032705006394E5006F000001370110F02B
:10022000130141F22320C101370110F0130101F243
:100230002320010013000000130000001300000041
:0C02400013000000130000001300000079
:040000058000006C0B
:00000001FF
